 getfldnm005

 Timestamp is 8541c616 (reproducible build file hash)

 Preferred load address is 0000000180000000

 Start         Length     Name                   Class
 0001:00000000 00003500H .text$mn                CODE
 0001:00003500 00000036H .text$mn$00             CODE
 0001:00003536 00000092H .text$x                 CODE
 0002:00000000 000001c8H .idata$5                DATA
 0002:000001c8 00000038H .00cfg                  DATA
 0002:00000200 00000008H .CRT$XCA                DATA
 0002:00000208 00000008H .CRT$XCZ                DATA
 0002:00000210 00000008H .CRT$XIA                DATA
 0002:00000218 00000008H .CRT$XIC                DATA
 0002:00000220 00000008H .CRT$XIZ                DATA
 0002:00000228 00000008H .CRT$XLA                DATA
 0002:00000230 00000008H .CRT$XLZ                DATA
 0002:00000238 00000008H .CRT$XPA                DATA
 0002:00000240 00000008H .CRT$XPZ                DATA
 0002:00000248 00000008H .CRT$XTA                DATA
 0002:00000250 00000010H .CRT$XTZ                DATA
 0002:00000258 00000000H .gehcont$y              DATA
 0002:00000258 00000000H .gfids$y                DATA
 0002:00000260 00002320H .rdata                  DATA
 0002:00002580 00000000H .rdata$CastGuardVftablesA DATA
 0002:00002580 00000000H .rdata$CastGuardVftablesC DATA
 0002:00002580 00000028H .rdata$T                DATA
 0002:000025a8 000000a8H .rdata$voltmd           DATA
 0002:00002650 00000318H .rdata$zzzdbg           DATA
 0002:00002968 00000008H .rtc$IAA                DATA
 0002:00002970 00000008H .rtc$IZZ                DATA
 0002:00002978 00000008H .rtc$TAA                DATA
 0002:00002980 00000008H .rtc$TZZ                DATA
 0002:00002988 00000004H .tls                    DATA
 0002:0000298c 00000004H .tls$                   DATA
 0002:00002990 00000008H .tls$ZZZ                DATA
 0002:00002998 00000328H .xdata                  DATA
 0002:00002cc0 0000039cH .edata                  DATA
 0002:0000305c 0000008cH .idata$2                DATA
 0002:000030e8 00000018H .idata$3                DATA
 0002:00003100 000001c8H .idata$4                DATA
 0002:000032c8 00000486H .idata$6                DATA
 0003:00000000 00000500H .data                   DATA
 0003:00000500 0001b238H .bss                    DATA
 0004:00000000 000003b4H .pdata                  DATA

  Address         Publics by Value              Rva+Base               Lib:Object

 0000:00000000       __AbsoluteZero             0000000000000000     <absolute>
 0000:00000000       ___safe_se_handler_count   0000000000000000     <absolute>
 0000:00000000       ___safe_se_handler_table   0000000000000000     <absolute>
 0000:00000000       __arm64x_extra_rfe_table   0000000000000000     <absolute>
 0000:00000000       __arm64x_extra_rfe_table_size 0000000000000000     <absolute>
 0000:00000000       __arm64x_native_entrypoint 0000000000000000     <absolute>
 0000:00000000       __arm64x_redirection_metadata 0000000000000000     <absolute>
 0000:00000000       __arm64x_redirection_metadata_count 0000000000000000     <absolute>
 0000:00000000       __dynamic_value_reloc_table 0000000000000000     <absolute>
 0000:00000000       __enclave_config           0000000000000000     <absolute>
 0000:00000000       __guard_check_icall_a64n_fptr 0000000000000000     <absolute>
 0000:00000000       __guard_eh_cont_count      0000000000000000     <absolute>
 0000:00000000       __guard_eh_cont_table      0000000000000000     <absolute>
 0000:00000000       __guard_fids_count         0000000000000000     <absolute>
 0000:00000000       __guard_fids_table         0000000000000000     <absolute>
 0000:00000000       __guard_iat_count          0000000000000000     <absolute>
 0000:00000000       __guard_iat_table          0000000000000000     <absolute>
 0000:00000000       __guard_longjmp_count      0000000000000000     <absolute>
 0000:00000000       __guard_longjmp_table      0000000000000000     <absolute>
 0000:00000000       __hybrid_auxiliary_iat     0000000000000000     <absolute>
 0000:00000000       __hybrid_auxiliary_iat_copy 0000000000000000     <absolute>
 0000:00000000       __hybrid_code_map          0000000000000000     <absolute>
 0000:00000000       __hybrid_code_map_count    0000000000000000     <absolute>
 0000:00000000       __x64_code_ranges_to_entry_points 0000000000000000     <absolute>
 0000:00000000       __x64_code_ranges_to_entry_points_count 0000000000000000     <absolute>
 0000:00000100       __guard_flags              0000000000000100     <absolute>
 0000:00000000       __ImageBase                0000000180000000     <linker-defined>
 0001:00000000       ?NewObject@JNIEnv_@@QEAAPEAV_jobject@@PEAV_jclass@@PEAU_jmethodID@@ZZ 0000000180001000 f i libgetfldnm005.obj
 0001:00000028       ?TranslateError@@YAPEBDW4jvmtiError@@@Z 0000000180001028 f   libgetfldnm005.obj
 0001:000002e0       ?nsk_jni_check_exception@@YAHPEAUJNIEnv_@@QEBDH@Z 00000001800012e0 f   libgetfldnm005.obj
 0001:00000424       ?nsk_jni_lverify@@YAHHPEAUJNIEnv_@@HQEBDH1ZZ 0000000180001424 f   libgetfldnm005.obj
 0001:000004c4       Agent_Initialize           00000001800014c4 f   libgetfldnm005.obj
 0001:000005c4       Agent_OnAttach             00000001800015c4 f   libgetfldnm005.obj
 0001:000005c4       Agent_OnLoad               00000001800015c4 f   libgetfldnm005.obj
 0001:000005cc       Java_nsk_jvmti_GetFieldName_getfldnm005_check 00000001800015cc f   libgetfldnm005.obj
 0001:000007f8       Java_nsk_jvmti_unit_FollowReferences_FollowRefObjects_addRefToVerify 00000001800017f8 f   libgetfldnm005.obj
 0001:000009d0       Java_nsk_jvmti_unit_FollowReferences_FollowRefObjects_getTag 00000001800019d0 f   libgetfldnm005.obj
 0001:00000a90       Java_nsk_jvmti_unit_FollowReferences_FollowRefObjects_resetRefsToVerify 0000000180001a90 f   libgetfldnm005.obj
 0001:00000a98       Java_nsk_jvmti_unit_FollowReferences_FollowRefObjects_resetTags 0000000180001a98 f   libgetfldnm005.obj
 0001:00000adc       Java_nsk_jvmti_unit_FollowReferences_FollowRefObjects_setTag 0000000180001adc f   libgetfldnm005.obj
 0001:00000d34       Java_nsk_share_jvmti_ArgumentHandler_getAgentOptionsString 0000000180001d34 f   libgetfldnm005.obj
 0001:00000de4       Java_nsk_share_jvmti_DebugeeClass_checkStatus 0000000180001de4 f   libgetfldnm005.obj
 0001:00000e6c       Java_nsk_share_jvmti_DebugeeClass_resetAgentData 0000000180001e6c f   libgetfldnm005.obj
 0001:00000ecc       Java_nsk_share_jvmti_RedefineAgent_agentStatus 0000000180001ecc f   libgetfldnm005.obj
 0001:00000ed8       Java_nsk_share_jvmti_RedefineAgent_isRedefined 0000000180001ed8 f   libgetfldnm005.obj
 0001:00000ee4       Java_nsk_share_jvmti_RedefineAgent_redefineAttempted 0000000180001ee4 f   libgetfldnm005.obj
 0001:00000ef0       MA_checkStatus             0000000180001ef0 f   libgetfldnm005.obj
 0001:00000f94       __local_stdio_printf_options 0000000180001f94 f i libgetfldnm005.obj
 0001:00001668       exitOnError                0000000180002668 f   libgetfldnm005.obj
 0001:0000171c       fprintf                    000000018000271c f i libgetfldnm005.obj
 0001:00001760       nsk_complain               0000000180002760 f   libgetfldnm005.obj
 0001:0000178c       nsk_jvmti_createJVMTIEnv   000000018000278c f   libgetfldnm005.obj
 0001:000018bc       nsk_jvmti_lverify          00000001800028bc f   libgetfldnm005.obj
 0001:000019ac       nsk_jvmti_parseOptions     00000001800029ac f   libgetfldnm005.obj
 0001:00001bfc       nsk_jvmti_resetAgentData   0000000180002bfc f   libgetfldnm005.obj
 0001:00001c7c       nsk_jvmti_setFailStatus    0000000180002c7c f   libgetfldnm005.obj
 0001:00001cb8       nsk_lcomplain              0000000180002cb8 f   libgetfldnm005.obj
 0001:00001cd8       nsk_ldisplay               0000000180002cd8 f   libgetfldnm005.obj
 0001:00001cf8       nsk_ltrace                 0000000180002cf8 f   libgetfldnm005.obj
 0001:00001d18       nsk_lvcomplain             0000000180002d18 f   libgetfldnm005.obj
 0001:00001ed0       nsk_lvdisplay              0000000180002ed0 f   libgetfldnm005.obj
 0001:00001f1c       nsk_lverify                0000000180002f1c f   libgetfldnm005.obj
 0001:00001f78       nsk_lvtrace                0000000180002f78 f   libgetfldnm005.obj
 0001:00001fd8       nsk_printf                 0000000180002fd8 f   libgetfldnm005.obj
 0001:00002000       nsk_vprintf                0000000180003000 f   libgetfldnm005.obj
 0001:000020b4       printf                     00000001800030b4 f i libgetfldnm005.obj
 0001:000025dc       __raise_securityfailure    00000001800035dc f   MSVCRT:gs_report.obj
 0001:00002610       __report_gsfailure         0000000180003610 f   MSVCRT:gs_report.obj
 0001:00002850       __GSHandlerCheck           0000000180003850 f   MSVCRT:gshandler.obj
 0001:00002870       __GSHandlerCheckCommon     0000000180003870 f   MSVCRT:gshandler.obj
 0001:000028e0       __security_check_cookie    00000001800038e0 f   MSVCRT:amdsecgs.obj
 0001:00002c20       _DllMainCRTStartup         0000000180003c20 f   MSVCRT:dll_dllmain.obj
 0001:00002c60       __scrt_acquire_startup_lock 0000000180003c60 f   MSVCRT:utility.obj
 0001:00002c9c       __scrt_dllmain_after_initialize_c 0000000180003c9c f   MSVCRT:utility.obj
 0001:00002cd0       __scrt_dllmain_before_initialize_c 0000000180003cd0 f   MSVCRT:utility.obj
 0001:00002ce8       __scrt_dllmain_crt_thread_attach 0000000180003ce8 f   MSVCRT:utility.obj
 0001:00002d10       __scrt_dllmain_crt_thread_detach 0000000180003d10 f   MSVCRT:utility.obj
 0001:00002d28       __scrt_dllmain_exception_filter 0000000180003d28 f   MSVCRT:utility.obj
 0001:00002d88       __scrt_dllmain_uninitialize_c 0000000180003d88 f   MSVCRT:utility.obj
 0001:00002db8       __scrt_dllmain_uninitialize_critical 0000000180003db8 f   MSVCRT:utility.obj
 0001:00002dcc       __scrt_initialize_crt      0000000180003dcc f   MSVCRT:utility.obj
 0001:00002e18       __scrt_initialize_onexit_tables 0000000180003e18 f   MSVCRT:utility.obj
 0001:00002ea4       __scrt_is_nonwritable_in_current_image 0000000180003ea4 f   MSVCRT:utility.obj
 0001:00002f3c       __scrt_release_startup_lock 0000000180003f3c f   MSVCRT:utility.obj
 0001:00002f60       __scrt_uninitialize_crt    0000000180003f60 f   MSVCRT:utility.obj
 0001:00002f8c       _onexit                    0000000180003f8c f   MSVCRT:utility.obj
 0001:00002fc8       atexit                     0000000180003fc8 f   MSVCRT:utility.obj
 0001:00002fe0       __crt_debugger_hook        0000000180003fe0 f   MSVCRT:utility_desktop.obj
 0001:00002fe8       __scrt_fastfail            0000000180003fe8 f   MSVCRT:utility_desktop.obj
 0001:00003134       _guard_check_icall_nop     0000000180004134 f i MSVCRT:guard_support.obj
 0001:00003138       __security_init_cookie     0000000180004138 f   MSVCRT:gs_support.obj
 0001:000031e4       DllMain                    00000001800041e4 f   MSVCRT:dll_dllmain_stub.obj
 0001:00003208       ?__scrt_initialize_type_info@@YAXXZ 0000000180004208 f   MSVCRT:tncleanup.obj
 0001:00003218       ?__scrt_uninitialize_type_info@@YAXXZ 0000000180004218 f   MSVCRT:tncleanup.obj
 0001:00003224       __local_stdio_scanf_options 0000000180004224 f i MSVCRT:default_local_stdio_options.obj
 0001:0000322c       __scrt_initialize_default_local_stdio_options 000000018000422c f   MSVCRT:default_local_stdio_options.obj
 0001:00003248       __scrt_get_dyn_tls_init_callback 0000000180004248 f   MSVCRT:dyn_tls_init.obj
 0001:00003250       _RTC_Initialize            0000000180004250 f   MSVCRT:initsect.obj
 0001:0000328c       _RTC_Terminate             000000018000428c f   MSVCRT:initsect.obj
 0001:000032c8       __isa_available_init       00000001800042c8 f   MSVCRT:cpu_disp.obj
 0001:00003474       _get_startup_argv_mode     0000000180004474 f   MSVCRT:argv_mode.obj
 0001:0000347c       __scrt_is_ucrt_dll_in_use  000000018000447c f   MSVCRT:ucrt_detection.obj
 0001:00003490       memcpy                     0000000180004490 f   vcruntime:VCRUNTIME140.dll
 0001:00003496       memset                     0000000180004496 f   vcruntime:VCRUNTIME140.dll
 0001:0000349c       strchr                     000000018000449c f   vcruntime:VCRUNTIME140.dll
 0001:000034a2       __C_specific_handler       00000001800044a2 f   vcruntime:VCRUNTIME140.dll
 0001:000034a8       __std_type_info_destroy_list 00000001800044a8 f   vcruntime:VCRUNTIME140.dll
 0001:000034ae       strcmp                     00000001800044ae f   ucrt:api-ms-win-crt-string-l1-1-0.dll
 0001:000034b4       strlen                     00000001800044b4 f   ucrt:api-ms-win-crt-string-l1-1-0.dll
 0001:000034ba       _initterm                  00000001800044ba f   ucrt:api-ms-win-crt-runtime-l1-1-0.dll
 0001:000034c0       _initterm_e                00000001800044c0 f   ucrt:api-ms-win-crt-runtime-l1-1-0.dll
 0001:000034c6       _seh_filter_dll            00000001800044c6 f   ucrt:api-ms-win-crt-runtime-l1-1-0.dll
 0001:000034cc       _configure_narrow_argv     00000001800044cc f   ucrt:api-ms-win-crt-runtime-l1-1-0.dll
 0001:000034d2       _initialize_narrow_environment 00000001800044d2 f   ucrt:api-ms-win-crt-runtime-l1-1-0.dll
 0001:000034d8       _initialize_onexit_table   00000001800044d8 f   ucrt:api-ms-win-crt-runtime-l1-1-0.dll
 0001:000034de       _register_onexit_function  00000001800044de f   ucrt:api-ms-win-crt-runtime-l1-1-0.dll
 0001:000034e4       _execute_onexit_table      00000001800044e4 f   ucrt:api-ms-win-crt-runtime-l1-1-0.dll
 0001:000034ea       _crt_atexit                00000001800044ea f   ucrt:api-ms-win-crt-runtime-l1-1-0.dll
 0001:000034f0       _cexit                     00000001800044f0 f   ucrt:api-ms-win-crt-runtime-l1-1-0.dll
 0001:000034f8       __acrt_initialize          00000001800044f8 f   MSVCRT:ucrt_stubs.obj
 0001:000034f8       __acrt_thread_attach       00000001800044f8 f   MSVCRT:ucrt_stubs.obj
 0001:000034f8       __acrt_thread_detach       00000001800044f8 f   MSVCRT:ucrt_stubs.obj
 0001:000034f8       __acrt_uninitialize        00000001800044f8 f   MSVCRT:ucrt_stubs.obj
 0001:000034f8       __acrt_uninitialize_critical 00000001800044f8 f   MSVCRT:ucrt_stubs.obj
 0001:000034f8       __scrt_stub_for_acrt_initialize 00000001800044f8 f   MSVCRT:ucrt_stubs.obj
 0001:000034f8       __scrt_stub_for_acrt_thread_attach 00000001800044f8 f   MSVCRT:ucrt_stubs.obj
 0001:000034f8       __scrt_stub_for_acrt_thread_detach 00000001800044f8 f   MSVCRT:ucrt_stubs.obj
 0001:000034f8       __scrt_stub_for_acrt_uninitialize 00000001800044f8 f   MSVCRT:ucrt_stubs.obj
 0001:000034f8       __scrt_stub_for_acrt_uninitialize_critical 00000001800044f8 f   MSVCRT:ucrt_stubs.obj
 0001:000034f8       __vcrt_initialize          00000001800044f8 f   MSVCRT:ucrt_stubs.obj
 0001:000034f8       __vcrt_thread_attach       00000001800044f8 f   MSVCRT:ucrt_stubs.obj
 0001:000034f8       __vcrt_thread_detach       00000001800044f8 f   MSVCRT:ucrt_stubs.obj
 0001:000034f8       __vcrt_uninitialize        00000001800044f8 f   MSVCRT:ucrt_stubs.obj
 0001:000034f8       __vcrt_uninitialize_critical 00000001800044f8 f   MSVCRT:ucrt_stubs.obj
 0001:000034fc       __scrt_stub_for_is_c_termination_complete 00000001800044fc f   MSVCRT:ucrt_stubs.obj
 0001:000034fc       _is_c_termination_complete 00000001800044fc f   MSVCRT:ucrt_stubs.obj
 0001:00003510       _guard_dispatch_icall_nop  0000000180004510 f   MSVCRT:guard_dispatch.obj
 0001:00003530       _guard_xfg_dispatch_icall_nop 0000000180004530 f   MSVCRT:guard_xfg_dispatch.obj
 0002:00000000       __imp_RtlCaptureContext    0000000180005000     kernel32:KERNEL32.dll
 0002:00000008       __imp_RtlLookupFunctionEntry 0000000180005008     kernel32:KERNEL32.dll
 0002:00000010       __imp_RtlVirtualUnwind     0000000180005010     kernel32:KERNEL32.dll
 0002:00000018       __imp_UnhandledExceptionFilter 0000000180005018     kernel32:KERNEL32.dll
 0002:00000020       __imp_SetUnhandledExceptionFilter 0000000180005020     kernel32:KERNEL32.dll
 0002:00000028       __imp_GetCurrentProcess    0000000180005028     kernel32:KERNEL32.dll
 0002:00000030       __imp_TerminateProcess     0000000180005030     kernel32:KERNEL32.dll
 0002:00000038       __imp_IsProcessorFeaturePresent 0000000180005038     kernel32:KERNEL32.dll
 0002:00000040       __imp_CloseHandle          0000000180005040     kernel32:KERNEL32.dll
 0002:00000048       __imp_InitializeCriticalSectionAndSpinCount 0000000180005048     kernel32:KERNEL32.dll
 0002:00000050       __imp_DeleteCriticalSection 0000000180005050     kernel32:KERNEL32.dll
 0002:00000058       __imp_CreateEventW         0000000180005058     kernel32:KERNEL32.dll
 0002:00000060       __imp_GetModuleHandleW     0000000180005060     kernel32:KERNEL32.dll
 0002:00000068       __imp_GetProcAddress       0000000180005068     kernel32:KERNEL32.dll
 0002:00000070       __imp_IsDebuggerPresent    0000000180005070     kernel32:KERNEL32.dll
 0002:00000078       __imp_QueryPerformanceCounter 0000000180005078     kernel32:KERNEL32.dll
 0002:00000080       __imp_GetCurrentProcessId  0000000180005080     kernel32:KERNEL32.dll
 0002:00000088       __imp_GetCurrentThreadId   0000000180005088     kernel32:KERNEL32.dll
 0002:00000090       __imp_GetSystemTimeAsFileTime 0000000180005090     kernel32:KERNEL32.dll
 0002:00000098       __imp_DisableThreadLibraryCalls 0000000180005098     kernel32:KERNEL32.dll
 0002:000000a0       __imp_InitializeSListHead  00000001800050a0     kernel32:KERNEL32.dll
 0002:000000a8       \177KERNEL32_NULL_THUNK_DATA 00000001800050a8     kernel32:KERNEL32.dll
 0002:000000b0       __imp_memcpy               00000001800050b0     vcruntime:VCRUNTIME140.dll
 0002:000000b8       __imp_memset               00000001800050b8     vcruntime:VCRUNTIME140.dll
 0002:000000c0       __imp_strchr               00000001800050c0     vcruntime:VCRUNTIME140.dll
 0002:000000c8       __imp___C_specific_handler 00000001800050c8     vcruntime:VCRUNTIME140.dll
 0002:000000d0       __imp___std_type_info_destroy_list 00000001800050d0     vcruntime:VCRUNTIME140.dll
 0002:000000d8       \177VCRUNTIME140_NULL_THUNK_DATA 00000001800050d8     vcruntime:VCRUNTIME140.dll
 0002:000000e0       __imp_strtol               00000001800050e0     ucrt:api-ms-win-crt-convert-l1-1-0.dll
 0002:000000e8       \177api-ms-win-crt-convert-l1-1-0_NULL_THUNK_DATA 00000001800050e8     ucrt:api-ms-win-crt-convert-l1-1-0.dll
 0002:000000f0       __imp_malloc               00000001800050f0     ucrt:api-ms-win-crt-heap-l1-1-0.dll
 0002:000000f8       __imp_free                 00000001800050f8     ucrt:api-ms-win-crt-heap-l1-1-0.dll
 0002:00000100       \177api-ms-win-crt-heap-l1-1-0_NULL_THUNK_DATA 0000000180005100     ucrt:api-ms-win-crt-heap-l1-1-0.dll
 0002:00000108       __imp__errno               0000000180005108     ucrt:api-ms-win-crt-runtime-l1-1-0.dll
 0002:00000110       __imp_exit                 0000000180005110     ucrt:api-ms-win-crt-runtime-l1-1-0.dll
 0002:00000118       __imp__cexit               0000000180005118     ucrt:api-ms-win-crt-runtime-l1-1-0.dll
 0002:00000120       __imp__crt_atexit          0000000180005120     ucrt:api-ms-win-crt-runtime-l1-1-0.dll
 0002:00000128       __imp__execute_onexit_table 0000000180005128     ucrt:api-ms-win-crt-runtime-l1-1-0.dll
 0002:00000130       __imp__register_onexit_function 0000000180005130     ucrt:api-ms-win-crt-runtime-l1-1-0.dll
 0002:00000138       __imp__initialize_onexit_table 0000000180005138     ucrt:api-ms-win-crt-runtime-l1-1-0.dll
 0002:00000140       __imp__initialize_narrow_environment 0000000180005140     ucrt:api-ms-win-crt-runtime-l1-1-0.dll
 0002:00000148       __imp__configure_narrow_argv 0000000180005148     ucrt:api-ms-win-crt-runtime-l1-1-0.dll
 0002:00000150       __imp__seh_filter_dll      0000000180005150     ucrt:api-ms-win-crt-runtime-l1-1-0.dll
 0002:00000158       __imp__initterm_e          0000000180005158     ucrt:api-ms-win-crt-runtime-l1-1-0.dll
 0002:00000160       __imp__initterm            0000000180005160     ucrt:api-ms-win-crt-runtime-l1-1-0.dll
 0002:00000168       \177api-ms-win-crt-runtime-l1-1-0_NULL_THUNK_DATA 0000000180005168     ucrt:api-ms-win-crt-runtime-l1-1-0.dll
 0002:00000170       __imp___acrt_iob_func      0000000180005170     ucrt:api-ms-win-crt-stdio-l1-1-0.dll
 0002:00000178       __imp_fflush               0000000180005178     ucrt:api-ms-win-crt-stdio-l1-1-0.dll
 0002:00000180       __imp___stdio_common_vsprintf 0000000180005180     ucrt:api-ms-win-crt-stdio-l1-1-0.dll
 0002:00000188       __imp___stdio_common_vfprintf 0000000180005188     ucrt:api-ms-win-crt-stdio-l1-1-0.dll
 0002:00000190       \177api-ms-win-crt-stdio-l1-1-0_NULL_THUNK_DATA 0000000180005190     ucrt:api-ms-win-crt-stdio-l1-1-0.dll
 0002:00000198       __imp_strcmp               0000000180005198     ucrt:api-ms-win-crt-string-l1-1-0.dll
 0002:000001a0       __imp__strdup              00000001800051a0     ucrt:api-ms-win-crt-string-l1-1-0.dll
 0002:000001a0       __imp_strdup               00000001800051a0     ucrt:api-ms-win-crt-string-l1-1-0.dll
 0002:000001a8       __imp_strlen               00000001800051a8     ucrt:api-ms-win-crt-string-l1-1-0.dll
 0002:000001b0       __imp_strpbrk              00000001800051b0     ucrt:api-ms-win-crt-string-l1-1-0.dll
 0002:000001b8       __imp_strncpy              00000001800051b8     ucrt:api-ms-win-crt-string-l1-1-0.dll
 0002:000001c0       \177api-ms-win-crt-string-l1-1-0_NULL_THUNK_DATA 00000001800051c0     ucrt:api-ms-win-crt-string-l1-1-0.dll
 0002:000001c8       __guard_check_icall_fptr   00000001800051c8     MSVCRT:guard_support.obj
 0002:000001d0       __guard_xfg_check_icall_fptr 00000001800051d0     MSVCRT:guard_support.obj
 0002:000001d8       __guard_dispatch_icall_fptr 00000001800051d8     MSVCRT:guard_support.obj
 0002:000001e0       __guard_xfg_dispatch_icall_fptr 00000001800051e0     MSVCRT:guard_support.obj
 0002:000001e8       __guard_xfg_table_dispatch_icall_fptr 00000001800051e8     MSVCRT:guard_support.obj
 0002:000001f0       __castguard_check_failure_os_handled_fptr 00000001800051f0     MSVCRT:guard_support.obj
 0002:000001f8       __guard_memcpy_fptr        00000001800051f8     vcruntime:softmemtag.obj
 0002:00000200       __xc_a                     0000000180005200     MSVCRT:initializers.obj
 0002:00000208       __xc_z                     0000000180005208     MSVCRT:initializers.obj
 0002:00000210       __xi_a                     0000000180005210     MSVCRT:initializers.obj
 0002:00000220       __xi_z                     0000000180005220     MSVCRT:initializers.obj
 0002:00000228       __xl_a                     0000000180005228     MSVCRT:tlssup.obj
 0002:00000230       __xl_z                     0000000180005230     MSVCRT:tlssup.obj
 0002:00000238       __xp_a                     0000000180005238     MSVCRT:initializers.obj
 0002:00000240       __xp_z                     0000000180005240     MSVCRT:initializers.obj
 0002:00000248       __xt_a                     0000000180005248     MSVCRT:initializers.obj
 0002:00000250       __xt_z                     0000000180005250     MSVCRT:initializers.obj
 0002:00000260       g_refKindStr               0000000180005260     libgetfldnm005.obj
 0002:00000410       ??_C@_09BPLDFGCI@unknown_0@ 0000000180005410     libgetfldnm005.obj
 0002:00000420       ??_C@_0BL@FPNMECJD@JVMTI_HEAP_REFERENCE_CLASS@ 0000000180005420     libgetfldnm005.obj
 0002:00000440       ??_C@_0BL@FKGKKLNM@JVMTI_HEAP_REFERENCE_FIELD@ 0000000180005440     libgetfldnm005.obj
 0002:00000460       ??_C@_0CD@CAEHCFJF@JVMTI_HEAP_REFERENCE_ARRAY_ELEM@ 0000000180005460     libgetfldnm005.obj
 0002:00000488       ??_C@_0CC@DNEBMCNK@JVMTI_HEAP_REFERENCE_CLASS_LOAD@ 0000000180005488     libgetfldnm005.obj
 0002:000004b0       ??_C@_0BN@CJMIPEBB@JVMTI_HEAP_REFERENCE_SIGNERS@ 00000001800054b0     libgetfldnm005.obj
 0002:000004d0       ??_C@_0CH@HBOIDPEB@JVMTI_HEAP_REFERENCE_PROTECTION@ 00000001800054d0     libgetfldnm005.obj
 0002:000004f8       ??_C@_0BP@MDKGDGKL@JVMTI_HEAP_REFERENCE_INTERFACE@ 00000001800054f8     libgetfldnm005.obj
 0002:00000518       ??_C@_0CC@JJMIHNJH@JVMTI_HEAP_REFERENCE_STATIC_FIE@ 0000000180005518     libgetfldnm005.obj
 0002:00000540       ??_C@_0CD@IDHEEGID@JVMTI_HEAP_REFERENCE_CONSTANT_P@ 0000000180005540     libgetfldnm005.obj
 0002:00000568       ??_C@_0CA@EFFCHNG@JVMTI_HEAP_REFERENCE_SUPERCLASS@ 0000000180005568     libgetfldnm005.obj
 0002:00000588       ??_C@_0L@PCDFHGCJ@unknown_11@ 0000000180005588     libgetfldnm005.obj
 0002:00000598       ??_C@_0L@NJBICFOK@unknown_12@ 0000000180005598     libgetfldnm005.obj
 0002:000005a8       ??_C@_0L@MAADBEKL@unknown_13@ 00000001800055a8     libgetfldnm005.obj
 0002:000005b8       ??_C@_0L@IPECICGM@unknown_14@ 00000001800055b8     libgetfldnm005.obj
 0002:000005c8       ??_C@_0L@JGFJLDCN@unknown_15@ 00000001800055c8     libgetfldnm005.obj
 0002:000005d8       ??_C@_0L@LNHEOAOO@unknown_16@ 00000001800055d8     libgetfldnm005.obj
 0002:000005e8       ??_C@_0L@KEGPNBKP@unknown_17@ 00000001800055e8     libgetfldnm005.obj
 0002:000005f8       ??_C@_0L@CDPHMNGA@unknown_18@ 00000001800055f8     libgetfldnm005.obj
 0002:00000608       ??_C@_0L@DKOMPMCB@unknown_19@ 0000000180005608     libgetfldnm005.obj
 0002:00000618       ??_C@_0L@OJGIPJDB@unknown_20@ 0000000180005618     libgetfldnm005.obj
 0002:00000628       ??_C@_0CA@KAOFNDEM@JVMTI_HEAP_REFERENCE_JNI_GLOBAL@ 0000000180005628     libgetfldnm005.obj
 0002:00000648       ??_C@_0CC@HPFAJBK@JVMTI_HEAP_REFERENCE_SYSTEM_CLA@ 0000000180005648     libgetfldnm005.obj
 0002:00000670       ??_C@_0BN@FDEGFOHC@JVMTI_HEAP_REFERENCE_MONITOR@ 0000000180005670     libgetfldnm005.obj
 0002:00000690       ??_C@_0CB@HKIBCMAJ@JVMTI_HEAP_REFERENCE_STACK_LOCA@ 0000000180005690     libgetfldnm005.obj
 0002:000006b8       ??_C@_0BP@EAACMMOE@JVMTI_HEAP_REFERENCE_JNI_LOCAL@ 00000001800056b8     libgetfldnm005.obj
 0002:000006d8       ??_C@_0BM@IJDEOGOE@JVMTI_HEAP_REFERENCE_THREAD@ 00000001800056d8     libgetfldnm005.obj
 0002:000006f8       ??_C@_0BL@EDGPPKC@JVMTI_HEAP_REFERENCE_OTHER@ 00000001800056f8     libgetfldnm005.obj
 0002:00000714       ??_C@_04BCJPDBDA@Code@     0000000180005714     libgetfldnm005.obj
 0002:00000720       ??_C@_0BA@OCLMCFKC@LineNumberTable@ 0000000180005720     libgetfldnm005.obj
 0002:00000730       ??_C@_0BD@CPAEPILC@LocalVariableTable@ 0000000180005730     libgetfldnm005.obj
 0002:00000748       ??_C@_0BH@NMBDNHBD@LocalVariableTypeTable@ 0000000180005748     libgetfldnm005.obj
 0002:00000760       ??_C@_0O@HIHEEDNJ@StackMapTable@ 0000000180005760     libgetfldnm005.obj
 0002:00000770       ??_C@_0P@DFIPEBLK@_getfldnm005St@ 0000000180005770     libgetfldnm005.obj
 0002:00000780       ??_C@_06GGHJAEBN@static@   0000000180005780     libgetfldnm005.obj
 0002:00000788       ??_C@_0CF@OLFABDJ@Lnsk?1jvmti?1GetFieldName?1getfldn@ 0000000180005788     libgetfldnm005.obj
 0002:000007b0       ??_C@_04MLLLIHIP@null@     00000001800057b0     libgetfldnm005.obj
 0002:000007b8       ??_C@_0O@KLNMPCLP@_getfldnm005b@ 00000001800057b8     libgetfldnm005.obj
 0002:000007c8       ??_C@_08EMNENPBA@instance@ 00000001800057c8     libgetfldnm005.obj
 0002:000007d8       ??_C@_0CG@NEMHAO@Lnsk?1jvmti?1GetFieldName?1getfldn@ 00000001800057d8     libgetfldnm005.obj
 0002:00000800       ??_C@_0DK@PFOIHCEL@Lnsk?1jvmti?1GetFieldName?1getfldn@ 0000000180005800     libgetfldnm005.obj
 0002:00000840       ??_C@_0BA@BFEHKGIA@_getfldnm005bSt@ 0000000180005840     libgetfldnm005.obj
 0002:00000850       ??_C@_0O@LCMHMDPO@_getfldnm005c@ 0000000180005850     libgetfldnm005.obj
 0002:00000860       ??_C@_0CG@BBGKNDJ@Lnsk?1jvmti?1GetFieldName?1getfldn@ 0000000180005860     libgetfldnm005.obj
 0002:00000890       ??_C@_0EO@KOIBDHHM@Lnsk?1jvmti?1GetFieldName?1getfldn@ 0000000180005890     libgetfldnm005.obj
 0002:000008e0       ??_C@_0BA@KNPLMBOF@_getfldnm005cSt@ 00000001800058e0     libgetfldnm005.obj
 0002:000008f0       ??_C@_0O@OEJNGEHI@_getfldnm005e@ 00000001800058f0     libgetfldnm005.obj
 0002:00000900       ??_C@_0CG@FJLNBIL@Lnsk?1jvmti?1GetFieldName?1getfldn@ 0000000180005900     libgetfldnm005.obj
 0002:00000928       ??_C@_0BA@IIJAJODJ@_getfldnm005eSt@ 0000000180005928     libgetfldnm005.obj
 0002:00000938       ??_C@_0P@GEIHFBCP@_getfldnm005if@ 0000000180005938     libgetfldnm005.obj
 0002:00000948       ??_C@_0CH@GIGPCMBK@Lnsk?1jvmti?1GetFieldName?1getfldn@ 0000000180005948     libgetfldnm005.obj
 0002:00000970       ??_C@_0DL@KEGNGGNL@Lnsk?1jvmti?1GetFieldName?1getfldn@ 0000000180005970     libgetfldnm005.obj
 0002:000009b0       ??_C@_0BB@CLNJBBJD@_getfldnm005ifSt@ 00000001800059b0     libgetfldnm005.obj
 0002:000009c8       ??_C@_0O@NGKLAGPK@_getfldnm005g@ 00000001800059c8     libgetfldnm005.obj
 0002:000009d8       ??_C@_0CG@GBPAFOF@Lnsk?1jvmti?1GetFieldName?1getfldn@ 00000001800059d8     libgetfldnm005.obj
 0002:00000a00       ??_C@_0EN@EKFNBAEB@Lnsk?1jvmti?1GetFieldName?1getfldn@ 0000000180005a00     libgetfldnm005.obj
 0002:00000a50       ??_C@_0BA@CCJJFGLC@_getfldnm005gSt@ 0000000180005a50     libgetfldnm005.obj
 0002:00000a60       ??_C@_0BB@MGNJLDCE@_getfldnm005gArr@ 0000000180005a60     libgetfldnm005.obj
 0002:00000a78       ??_C@_0CH@CJDIDCEI@?$FLLnsk?1jvmti?1GetFieldName?1getfld@ 0000000180005a78     libgetfldnm005.obj
 0002:00000aa0       ??_C@_0L@HCDIAMJG@?9?5?$CFs?0?5?$CFd?3?5@ 0000000180005aa0     libgetfldnm005.obj
 0002:00000ab0       ??_C@_0JI@HLPECLFI@?$CD?5?4?4?4?6?$CD?5ERROR?3?5too?5many?5complai@ 0000000180005ab0     libgetfldnm005.obj
 0002:00000b50       ??_C@_0ED@JNEKCCOB@The?5following?5fake?5exception?5st@ 0000000180005b50     libgetfldnm005.obj
 0002:00000b98       ??_C@_0CN@FCNMDFBH@nsk?4share?4Fake_Exception_for_RU@ 0000000180005b98     libgetfldnm005.obj
 0002:00000bc8       ??_C@_08PGFFNAEI@?$CI?$CFs?3?$CFd?$CJ?5@ 0000000180005bc8     libgetfldnm005.obj
 0002:00000bd8       ??_C@_0DP@IENMAEGI@s?2test?2hotspot?2jtreg?2vmTestbase@ 0000000180005bd8     libgetfldnm005.obj
 0002:00000c18       ??_C@_0BL@NDJLFFJB@?7at?5nsk_lvcomplain?$CI?$CFs?3?$CFd?$CJ?6@ 0000000180005c18     libgetfldnm005.obj
 0002:00000c38       ??_C@_0BC@JOOKAFKF@?$CD?5ERROR?3?5?$CFs?0?5?$CFd?3?5@ 0000000180005c38     libgetfldnm005.obj
 0002:00000c50       ??_C@_09KJEAHMEH@?$CD?5ERROR?3?5@ 0000000180005c50     libgetfldnm005.obj
 0002:00000c5c       ??_C@_02GPIOPFAK@?$DO?$DO@ 0000000180005c5c     libgetfldnm005.obj
 0002:00000c60       ??_C@_02FODMEDOG@?$DM?$DM@ 0000000180005c60     libgetfldnm005.obj
 0002:00000c64       ??_C@_02DJGKEECL@?4?4@     0000000180005c64     libgetfldnm005.obj
 0002:00000c68       ??_C@_0O@CJPGJOAF@?9?5?$CFs?0?5?$CFd?3?5?$CFs?5@ 0000000180005c68     libgetfldnm005.obj
 0002:00000c78       ??_C@_0CB@IAKPDOIC@?$CD?5?5?5verified?5assertion?5is?5FALSE@ 0000000180005c78     libgetfldnm005.obj
 0002:00000ca0       ??_C@_0CO@LGONDEPD@stdout?3?5fflush?5failed?5?9?5err?$DN?$CFd?5@ 0000000180005ca0     libgetfldnm005.obj
 0002:00000cd0       ??_C@_0CO@KBGKJPBD@stderr?3?5fflush?5failed?5?9?5err?$DN?$CFd?5@ 0000000180005cd0     libgetfldnm005.obj
 0002:00000d00       ??_C@_0BB@JCNMKLLK@JVMTI_ERROR_NONE@ 0000000180005d00     libgetfldnm005.obj
 0002:00000d18       ??_C@_0BL@LDIMKLPH@JVMTI_ERROR_INVALID_THREAD@ 0000000180005d18     libgetfldnm005.obj
 0002:00000d38       ??_C@_0CB@PJFPAIKJ@JVMTI_ERROR_INVALID_THREAD_GROU@ 0000000180005d38     libgetfldnm005.obj
 0002:00000d60       ??_C@_0BN@LLMKHMNF@JVMTI_ERROR_INVALID_PRIORITY@ 0000000180005d60     libgetfldnm005.obj
 0002:00000d80       ??_C@_0CB@MBOFKAGB@JVMTI_ERROR_THREAD_NOT_SUSPENDE@ 0000000180005d80     libgetfldnm005.obj
 0002:00000da8       ??_C@_0BN@FABOLPBI@JVMTI_ERROR_THREAD_SUSPENDED@ 0000000180005da8     libgetfldnm005.obj
 0002:00000dc8       ??_C@_0BN@FDGNOBJM@JVMTI_ERROR_THREAD_NOT_ALIVE@ 0000000180005dc8     libgetfldnm005.obj
 0002:00000de8       ??_C@_0BL@GOBIFKNJ@JVMTI_ERROR_INVALID_OBJECT@ 0000000180005de8     libgetfldnm005.obj
 0002:00000e08       ??_C@_0BK@FCMAJPPC@JVMTI_ERROR_INVALID_CLASS@ 0000000180005e08     libgetfldnm005.obj
 0002:00000e28       ??_C@_0BP@IKLLBKEB@JVMTI_ERROR_CLASS_NOT_PREPARED@ 0000000180005e28     libgetfldnm005.obj
 0002:00000e48       ??_C@_0BN@KLPPLKG@JVMTI_ERROR_INVALID_METHODID@ 0000000180005e48     libgetfldnm005.obj
 0002:00000e68       ??_C@_0BN@BCEKOKND@JVMTI_ERROR_INVALID_LOCATION@ 0000000180005e68     libgetfldnm005.obj
 0002:00000e88       ??_C@_0BM@DFDGPME@JVMTI_ERROR_INVALID_FIELDID@ 0000000180005e88     libgetfldnm005.obj
 0002:00000ea8       ??_C@_0BL@NELIEPEC@JVMTI_ERROR_NO_MORE_FRAMES@ 0000000180005ea8     libgetfldnm005.obj
 0002:00000ec8       ??_C@_0BJ@BDBECFDM@JVMTI_ERROR_OPAQUE_FRAME@ 0000000180005ec8     libgetfldnm005.obj
 0002:00000ee8       ??_C@_0BK@MIIFNLOB@JVMTI_ERROR_TYPE_MISMATCH@ 0000000180005ee8     libgetfldnm005.obj
 0002:00000f08       ??_C@_0BJ@HPCAOILC@JVMTI_ERROR_INVALID_SLOT@ 0000000180005f08     libgetfldnm005.obj
 0002:00000f28       ??_C@_0BG@CHILOPNI@JVMTI_ERROR_DUPLICATE@ 0000000180005f28     libgetfldnm005.obj
 0002:00000f40       ??_C@_0BG@DIEMLHKM@JVMTI_ERROR_NOT_FOUND@ 0000000180005f40     libgetfldnm005.obj
 0002:00000f58       ??_C@_0BM@NHMCKHOB@JVMTI_ERROR_INVALID_MONITOR@ 0000000180005f58     libgetfldnm005.obj
 0002:00000f78       ??_C@_0BO@PPEDAJGL@JVMTI_ERROR_NOT_MONITOR_OWNER@ 0000000180005f78     libgetfldnm005.obj
 0002:00000f98       ??_C@_0BG@FCAIPEID@JVMTI_ERROR_INTERRUPT@ 0000000180005f98     libgetfldnm005.obj
 0002:00000fb0       ??_C@_0CB@EGDBNKOI@JVMTI_ERROR_INVALID_CLASS_FORMA@ 0000000180005fb0     libgetfldnm005.obj
 0002:00000fd8       ??_C@_0CG@DGKOGIAL@JVMTI_ERROR_CIRCULAR_CLASS_DEFI@ 0000000180005fd8     libgetfldnm005.obj
 0002:00001000       ??_C@_0BP@ICEALPKC@JVMTI_ERROR_FAILS_VERIFICATION@ 0000000180006000     libgetfldnm005.obj
 0002:00001020       ??_C@_0DC@JDACLMIO@JVMTI_ERROR_UNSUPPORTED_REDEFIN@ 0000000180006020     libgetfldnm005.obj
 0002:00001058       ??_C@_0DE@GKDKNOMJ@JVMTI_ERROR_UNSUPPORTED_REDEFIN@ 0000000180006058     libgetfldnm005.obj
 0002:00001090       ??_C@_0BO@LAFKIOG@JVMTI_ERROR_INVALID_TYPESTATE@ 0000000180006090     libgetfldnm005.obj
 0002:000010b0       ??_C@_0DH@INDGCLLB@JVMTI_ERROR_UNSUPPORTED_REDEFIN@ 00000001800060b0     libgetfldnm005.obj
 0002:000010e8       ??_C@_0DE@NHEOMMGI@JVMTI_ERROR_UNSUPPORTED_REDEFIN@ 00000001800060e8     libgetfldnm005.obj
 0002:00001120       ??_C@_0CA@EKPNJOEP@JVMTI_ERROR_UNSUPPORTED_VERSION@ 0000000180006120     libgetfldnm005.obj
 0002:00001140       ??_C@_0BN@OFFMAHHL@JVMTI_ERROR_NAMES_DONT_MATCH@ 0000000180006140     libgetfldnm005.obj
 0002:00001160       ??_C@_0DN@HHBBLAKE@JVMTI_ERROR_UNSUPPORTED_REDEFIN@ 0000000180006160     libgetfldnm005.obj
 0002:000011a0       ??_C@_0DO@HMBGBGNA@JVMTI_ERROR_UNSUPPORTED_REDEFIN@ 00000001800061a0     libgetfldnm005.obj
 0002:000011e0       ??_C@_0BP@PBECGKHJ@JVMTI_ERROR_UNMODIFIABLE_CLASS@ 00000001800061e0     libgetfldnm005.obj
 0002:00001200       ??_C@_0BK@CANILEHF@JVMTI_ERROR_NOT_AVAILABLE@ 0000000180006200     libgetfldnm005.obj
 0002:00001220       ??_C@_0CE@INJKMEFK@JVMTI_ERROR_MUST_POSSESS_CAPABI@ 0000000180006220     libgetfldnm005.obj
 0002:00001248       ??_C@_0BJ@LBFPFPDM@JVMTI_ERROR_NULL_POINTER@ 0000000180006248     libgetfldnm005.obj
 0002:00001268       ??_C@_0BP@CHJPNNEM@JVMTI_ERROR_ABSENT_INFORMATION@ 0000000180006268     libgetfldnm005.obj
 0002:00001288       ??_C@_0BP@OMFMNLC@JVMTI_ERROR_INVALID_EVENT_TYPE@ 0000000180006288     libgetfldnm005.obj
 0002:000012a8       ??_C@_0BN@BIBNPHHO@JVMTI_ERROR_ILLEGAL_ARGUMENT@ 00000001800062a8     libgetfldnm005.obj
 0002:000012c8       ??_C@_0BK@KKNDHDCE@JVMTI_ERROR_NATIVE_METHOD@ 00000001800062c8     libgetfldnm005.obj
 0002:000012e8       ??_C@_0BK@PMKCFHAE@JVMTI_ERROR_OUT_OF_MEMORY@ 00000001800062e8     libgetfldnm005.obj
 0002:00001308       ??_C@_0BK@NNJBDMNB@JVMTI_ERROR_ACCESS_DENIED@ 0000000180006308     libgetfldnm005.obj
 0002:00001328       ??_C@_0BI@GHECLMNC@JVMTI_ERROR_WRONG_PHASE@ 0000000180006328     libgetfldnm005.obj
 0002:00001340       ??_C@_0BF@OLIHJOII@JVMTI_ERROR_INTERNAL@ 0000000180006340     libgetfldnm005.obj
 0002:00001358       ??_C@_0BO@EOHGKJHI@JVMTI_ERROR_UNATTACHED_THREAD@ 0000000180006358     libgetfldnm005.obj
 0002:00001378       ??_C@_0CA@LKHFDACL@JVMTI_ERROR_INVALID_ENVIRONMENT@ 0000000180006378     libgetfldnm005.obj
 0002:00001398       ??_C@_0BA@MMFHLOKK@?$DMunknown?5error?$DO@ 0000000180006398     libgetfldnm005.obj
 0002:000013a8       ??_C@_0CF@CBHOKDB@throwable?5?$DN?5jni?9?$DOExceptionOccur@ 00000001800063a8     libgetfldnm005.obj
 0002:000013d0       ??_C@_03OFAPEBGM@?$CFs?6@  00000001800063d0     libgetfldnm005.obj
 0002:000013d8       ??_C@_0DM@LPIGEGNJ@s?2test?2hotspot?2jtreg?2vmTestbase@ 00000001800063d8     libgetfldnm005.obj
 0002:00001418       ??_C@_0CC@NFCNPEPK@Exception?5in?5JNI?5call?5?$CIcleared?$CJ@ 0000000180006418     libgetfldnm005.obj
 0002:00001440       ??_C@_0BJ@IBAKFIKF@jni?9?$DOExceptionDescribe?$CI?$CJ@ 0000000180006440     libgetfldnm005.obj
 0002:00001460       ??_C@_0BG@GGKALKMH@jni?9?$DOExceptionClear?$CI?$CJ@ 0000000180006460     libgetfldnm005.obj
 0002:00001478       ??_C@_0CF@JMGFGJLJ@?$CD?5?5?5verified?5JNI?5assertion?5is?5F@ 0000000180006478     libgetfldnm005.obj
 0002:000014a0       ??_C@_07KBAMPNJK@verbose@  00000001800064a0     libgetfldnm005.obj
 0002:000014a8       ??_C@_0DN@PKJBOLAP@nsk_jvmti_parseOptions?$CI?$CJ?3?5unexp@ 00000001800064a8     libgetfldnm005.obj
 0002:000014e8       ??_C@_05IMBNNINJ@trace@    00000001800064e8     libgetfldnm005.obj
 0002:000014f0       ??_C@_0DD@BJKGNDMB@nsk_jvmti_parseOptions?$CI?$CJ?3?5no?5va@ 00000001800064f0     libgetfldnm005.obj
 0002:00001524       ??_C@_04CGFJFPFD@none@     0000000180006524     libgetfldnm005.obj
 0002:0000152c       ??_C@_06BMELKFMA@before@   000000018000652c     libgetfldnm005.obj
 0002:00001534       ??_C@_05CMKPCFDK@after@    0000000180006534     libgetfldnm005.obj
 0002:0000153c       ??_C@_03NFKEKGGK@all@      000000018000653c     libgetfldnm005.obj
 0002:00001540       ??_C@_0DM@NDNJGJKE@nsk_jvmti_parseOptions?$CI?$CJ?3?5uexpe@ 0000000180006540     libgetfldnm005.obj
 0002:00001580       ??_C@_08NBBJKJO@waittime@  0000000180006580     libgetfldnm005.obj
 0002:00001590       ??_C@_0DO@CMHGAOHC@nsk_jvmti_parseOptions?$CI?$CJ?3?5not?5i@ 0000000180006590     libgetfldnm005.obj
 0002:000015d0       ??_C@_0DL@LNMPBDLN@nsk_jvmti_parseOptions?$CI?$CJ?3?5negat@ 00000001800065d0     libgetfldnm005.obj
 0002:00001610       ??_C@_0DA@GMFJNOJH@nsk_jvmti_parseOptions?$CI?$CJ?3?5unkno@ 0000000180006610     libgetfldnm005.obj
 0002:00001640       ??_C@_0CO@CCIAMEAN@nsk_jvmti_parseOptions?$CI?$CJ?3?5found@ 0000000180006640     libgetfldnm005.obj
 0002:00001670       ??_C@_0CJ@OEGPCGDL@nsk_jvmti_parseOptions?$CI?$CJ?3?5out?5o@ 0000000180006670     libgetfldnm005.obj
 0002:000016a0       ??_C@_0DI@NMBHPGGF@nsk_jvmti_parseOptions?$CI?$CJ?3?5too?5m@ 00000001800066a0     libgetfldnm005.obj
 0002:000016d8       ??_C@_03POGCGECB@?5?0?$HO@ 00000001800066d8     libgetfldnm005.obj
 0002:000016e0       ??_C@_0CB@MLNJNCLJ@?5?5jvmti?5error?3?5code?$DN?$CFd?0?5name?$DN?$CFs@ 00000001800066e0     libgetfldnm005.obj
 0002:00001708       ??_C@_0CD@OHBGDKMK@?$CD?5?5?5jvmti?5error?3?5code?$DN?$CFd?0?5name?$DN@ 0000000180006708     libgetfldnm005.obj
 0002:00001730       ??_C@_0CG@JNNCGPHB@?$CD?5?5?5error?5expected?3?5code?$DN?$CFd?0?5na@ 0000000180006730     libgetfldnm005.obj
 0002:00001760       ??_C@_0EB@IMGKPCGE@?$CIstr_obj?5?$DN?5jni?9?$DONewStringUTF?$CIco@ 0000000180006760     libgetfldnm005.obj
 0002:000017b0       ??_C@_0EA@HFOGGBCC@s?2test?2hotspot?2jtreg?2vmTestbase@ 00000001800067b0     libgetfldnm005.obj
 0002:000017f0       ??_C@_05KKCIMGE@error@     00000001800067f0     libgetfldnm005.obj
 0002:000017f8       ??_C@_0CJ@JACLEAA@Test?5failed?5by?5setFailStatus?$CI?$CJ?4@ 00000001800067f8     libgetfldnm005.obj
 0002:00001828       ??_C@_0BD@HGNAOMCP@agent_data_monitor@ 0000000180006828     libgetfldnm005.obj
 0002:00001840       ??_C@_0EB@OGCLGKLN@javaVM?9?$DOGetEnv?$CI?$CIvoid?5?$CK?$CK?$CJ?$CGjvmti_@ 0000000180006840     libgetfldnm005.obj
 0002:00001890       ??_C@_0EA@PNBCDMOA@s?2test?2hotspot?2jtreg?2vmTestbase@ 0000000180006890     libgetfldnm005.obj
 0002:000018d0       ??_C@_0CI@DDPIFBGM@init_agent_data?$CIjvmti_env?0?5?$CGage@ 00000001800068d0     libgetfldnm005.obj
 0002:000018f8       ??_C@_0DI@ILAHDLMP@?$CI?$CKagentThreadProc?$CJ?$CIjvmti_env?0?5a@ 00000001800068f8     libgetfldnm005.obj
 0002:00001930       ??_C@_0BD@KDBALNLB@JVMTI?5agent?5thread@ 0000000180006930     libgetfldnm005.obj
 0002:00001948       ??_C@_0BB@NOKBFPFO@java?1lang?1Thread@ 0000000180006948     libgetfldnm005.obj
 0002:0000195c       ??_C@_06FALKBLGB@?$DMinit?$DO@ 000000018000695c     libgetfldnm005.obj
 0002:00001968       ??_C@_0BG@IKDDPPGD@?$CILjava?1lang?1String?$DL?$CJV@ 0000000180006968     libgetfldnm005.obj
 0002:00001980       ??_C@_0EB@IFJBFEKC@?$CIthreadClass?5?$DN?5jni_env?9?$DOFindCla@ 0000000180006980     libgetfldnm005.obj
 0002:000019d0       ??_C@_0GF@FGFIBKKL@?$CIthreadCtor?5?$DN?5jni_env?9?$DOGetMetho@ 00000001800069d0     libgetfldnm005.obj
 0002:00001a38       ??_C@_0DN@NCPDJLOG@?$CIthreadName?5?$DN?5jni_env?9?$DONewStrin@ 0000000180006a38     libgetfldnm005.obj
 0002:00001a80       ??_C@_0FE@PFKODBGC@?$CIthreadObject?5?$DN?5jni_env?9?$DONewObj@ 0000000180006a80     libgetfldnm005.obj
 0002:00001ae0       ??_C@_0ED@HOBAHHJI@?$CIthreadGlobalRef?5?$DN?5jni_env?9?$DONew@ 0000000180006ae0     libgetfldnm005.obj
 0002:00001b30       ??_C@_0FN@HNJJAHFC@jvmti_env?9?$DORunAgentThread?$CIagent@ 0000000180006b30     libgetfldnm005.obj
 0002:00001b90       ??_C@_0EA@MOJDNKDF@Debuggee?5status?5sync?5aborted?5be@ 0000000180006b90     libgetfldnm005.obj
 0002:00001bd0       ??_C@_0EA@EEOEJAEN@status?5?$DN?5syncDebuggeeStatus?$CIjni@ 0000000180006bd0     libgetfldnm005.obj
 0002:00001c10       ??_C@_0BL@JBCFNBMB@nsk_jvmti_resetAgentData?$CI?$CJ@ 0000000180006c10     libgetfldnm005.obj
 0002:00001c30       ??_C@_0EL@LPBEELIP@s?2test?2hotspot?2jtreg?2vmTestbase@ 0000000180006c30     libgetfldnm005.obj
 0002:00001c80       ??_C@_0CK@JDAMFDMJ@jvmti?9?$DOSetTag?$CIo?0?5tag?$CJ?5?$DN?$DN?5JVMTI_@ 0000000180006c80     libgetfldnm005.obj
 0002:00001cb0       ??_C@_0CC@DAMNHKNI@Can?8t?5set?5tag?5?$CFli?5for?5object?5?$CFl@ 0000000180006cb0     libgetfldnm005.obj
 0002:00001cd8       ??_C@_0DL@HAJPNKEF@jvmti?9?$DOGetObjectHashCode?$CIo?0?5?$CGha@ 0000000180006cd8     libgetfldnm005.obj
 0002:00001d18       ??_C@_0BL@JFPIEOBF@Can?8t?5get?5hash?5object?5?$CFlx?6@ 0000000180006d18     libgetfldnm005.obj
 0002:00001d38       ??_C@_0BG@DICPHBKN@setTag?3?5?$CF08x?5?$DM?9?5?$CF?53li@ 0000000180006d38     libgetfldnm005.obj
 0002:00001d50       ??_C@_0DH@FCEEBDMJ@?$CIs?5?$DN?5jni?9?$DOGetStringUTFChars?$CIsIn@ 0000000180006d50     libgetfldnm005.obj
 0002:00001d88       ??_C@_0BJ@OKKGHDCN@Can?8t?5get?5string?5at?5?$CF?$CDp?6@ 0000000180006d88     libgetfldnm005.obj
 0002:00001da8       ??_C@_0BP@EKFLGGFJ@Can?8t?5get?5string?5at?5?$CF?$CDp?3?5null?6@ 0000000180006da8     libgetfldnm005.obj
 0002:00001dc8       ??_C@_06ICODBHCL@?5?1?1?5?$CFs@ 0000000180006dc8     libgetfldnm005.obj
 0002:00001dd0       ??_C@_0DB@KGFPLEGO@?$CIr?5?$DN?5jvmti?9?$DOGetTag?$CIo?0?5?$CGtag?$CJ?$CJ?5?$DN?$DN@ 0000000180006dd0     libgetfldnm005.obj
 0002:00001e08       ??_C@_0CO@PDAGBCGJ@Can?8t?5GetTag?5for?5object?5?$CFlx?4?5Re@ 0000000180006e08     libgetfldnm005.obj
 0002:00001e38       ??_C@_0CH@HPEODOHC@TEST_BUG?3?5Max?4?5number?5of?5refs?5r@ 0000000180006e38     libgetfldnm005.obj
 0002:00001e60       ??_C@_0DI@PHFCABIM@?$CIr?5?$DN?5jvmti?9?$DOGetTag?$CIfrom?0?5?$CGtagFr@ 0000000180006e60     libgetfldnm005.obj
 0002:00001e98       ??_C@_0DI@MDEGFNKD@TEST_BUG?3?5Can?8t?5GetTag?5for?5obje@ 0000000180006e98     libgetfldnm005.obj
 0002:00001ed0       ??_C@_0DE@MLELJAHM@?$CIr?5?$DN?5jvmti?9?$DOGetTag?$CIto?0?5?$CGtagTo?$CJ?$CJ@ 0000000180006ed0     libgetfldnm005.obj
 0002:00001f10       ??_C@_0ED@FEDPOGLP@jvmti?9?$DOGetFieldName?$CItestedCls?0?5@ 0000000180006f10     libgetfldnm005.obj
 0002:00001f60       ??_C@_0FD@FJGIJMIG@s?2test?2hotspot?2jtreg?2vmTestbase@ 0000000180006f60     libgetfldnm005.obj
 0002:00001fb8       ??_C@_0DN@HHACFAK@TEST?5FAILED?3?5unable?5to?5get?5fiel@ 0000000180006fb8     libgetfldnm005.obj
 0002:00001ff8       ??_C@_0CC@LMBOAPAI@Checking?5signatures?5for?5?$CC?$CFs?$CC?5?4?4@ 0000000180006ff8     libgetfldnm005.obj
 0002:00002020       ??_C@_0GD@EGOLJDCK@TEST?5FAILED?3?5?$CFs?5field?5?$CC?$CFs?$CC?5has?6@ 0000000180007020     libgetfldnm005.obj
 0002:00002088       ??_C@_0DJ@ILKHGAIK@CHECK?5PASSED?3?5signature?3?5?$CC?$CFs?$CC?0?6@ 0000000180007088     libgetfldnm005.obj
 0002:000020c8       ??_C@_0CG@BGNDDPIG@Deallocating?5name?5?$CG?5signature?5a@ 00000001800070c8     libgetfldnm005.obj
 0002:000020f0       ??_C@_0CJ@LKCJEAJA@jvmti?9?$DODeallocate?$CI?$CIunsigned?5cha@ 00000001800070f0     libgetfldnm005.obj
 0002:00002120       ??_C@_0CJ@FGPJBFJB@jvmti?9?$DODeallocate?$CI?$CIunsigned?5cha@ 0000000180007120     libgetfldnm005.obj
 0002:00002150       ??_C@_0CN@BIIEKGPC@jvmti?9?$DODeallocate?$CI?$CIunsigned?5cha@ 0000000180007150     libgetfldnm005.obj
 0002:00002180       ??_C@_0BO@DMPDBABE@?$DO?$DO?$DO?5Finding?5?$CFs?5field?3?5?$CFs?5?4?4?4?6@ 0000000180007180     libgetfldnm005.obj
 0002:000021a0       ??_C@_0EP@PHDLICJD@?$CItestedFld?5?$DN?5jni?9?$DOGetFieldID?$CIob@ 00000001800071a0     libgetfldnm005.obj
 0002:000021f0       ??_C@_0DA@PGKKHOPB@TEST?5FAILERE?3?5unable?5to?5get?5fie@ 00000001800071f0     libgetfldnm005.obj
 0002:00002220       ??_C@_0FF@KBLKACEB@?$CItestedFld?5?$DN?5jni?9?$DOGetStaticFiel@ 0000000180007220     libgetfldnm005.obj
 0002:00002278       ??_C@_0BI@JPFOBOBH@?7?4?4?4?5got?5fieldID?3?50x?$CFp?6@ 0000000180007278     libgetfldnm005.obj
 0002:00002290       ??_C@_04DAGPOOAC@?$DM?$DM?$DM?6@ 0000000180007290     libgetfldnm005.obj
 0002:00002298       ??_C@_0CA@MNKGCBCG@nsk_jvmti_parseOptions?$CIoptions?$CJ@ 0000000180007298     libgetfldnm005.obj
 0002:000022b8       ??_C@_0DN@MIAMNFPH@?$CIjvmti?5?$DN?5nsk_jvmti_createJVMTIE@ 00000001800072b8     libgetfldnm005.obj
 0002:00002310       ??_C@_1EC@JIJBPKFM@?$AAa?$AAp?$AAi?$AA?9?$AAm?$AAs?$AA?9?$AAw?$AAi?$AAn?$AA?9?$AAc?$AAo?$AAr?$AAe@ 0000000180007310     MSVCRT:thread_safe_statics.obj
 0002:00002358       ??_C@_1BK@MGMFAEKH@?$AAk?$AAe?$AAr?$AAn?$AAe?$AAl?$AA3?$AA2?$AA?4?$AAd?$AAl?$AAl@ 0000000180007358     MSVCRT:thread_safe_statics.obj
 0002:00002378       ??_C@_0BJ@JEBJOJFJ@SleepConditionVariableCS@ 0000000180007378     MSVCRT:thread_safe_statics.obj
 0002:00002398       ??_C@_0BJ@PGPPEPCC@WakeAllConditionVariable@ 0000000180007398     MSVCRT:thread_safe_statics.obj
 0002:000023b8       _pDefaultRawDllMain        00000001800073b8     MSVCRT:dll_dllmain.obj
 0002:000023b8       _pRawDllMain               00000001800073b8     MSVCRT:dll_dllmain.obj
 0002:000023c0       __xmm@ffffffffffffffffffffffffffffffff 00000001800073c0     MSVCRT:utility.obj
 0002:000023d0       _load_config_used          00000001800073d0     MSVCRT:loadcfg.obj
 0002:00002580       _tls_used                  0000000180007580     MSVCRT:tlssup.obj
 0002:000025a8       __volatile_metadata        00000001800075a8     <linker-defined>
 0002:00002968       __rtc_iaa                  0000000180007968     MSVCRT:initsect.obj
 0002:00002970       __rtc_izz                  0000000180007970     MSVCRT:initsect.obj
 0002:00002978       __rtc_taa                  0000000180007978     MSVCRT:initsect.obj
 0002:00002980       __rtc_tzz                  0000000180007980     MSVCRT:initsect.obj
 0002:00002988       _tls_start                 0000000180007988     MSVCRT:tlssup.obj
 0002:0000298c       _Init_thread_epoch         000000018000798c     MSVCRT:thread_safe_statics.obj
 0002:00002990       _tls_end                   0000000180007990     MSVCRT:tlssup.obj
 0002:0000305c       __IMPORT_DESCRIPTOR_KERNEL32 000000018000805c     kernel32:KERNEL32.dll
 0002:00003070       __IMPORT_DESCRIPTOR_VCRUNTIME140 0000000180008070     vcruntime:VCRUNTIME140.dll
 0002:00003084       __IMPORT_DESCRIPTOR_api-ms-win-crt-heap-l1-1-0 0000000180008084     ucrt:api-ms-win-crt-heap-l1-1-0.dll
 0002:00003098       __IMPORT_DESCRIPTOR_api-ms-win-crt-runtime-l1-1-0 0000000180008098     ucrt:api-ms-win-crt-runtime-l1-1-0.dll
 0002:000030ac       __IMPORT_DESCRIPTOR_api-ms-win-crt-convert-l1-1-0 00000001800080ac     ucrt:api-ms-win-crt-convert-l1-1-0.dll
 0002:000030c0       __IMPORT_DESCRIPTOR_api-ms-win-crt-stdio-l1-1-0 00000001800080c0     ucrt:api-ms-win-crt-stdio-l1-1-0.dll
 0002:000030d4       __IMPORT_DESCRIPTOR_api-ms-win-crt-string-l1-1-0 00000001800080d4     ucrt:api-ms-win-crt-string-l1-1-0.dll
 0002:000030e8       __NULL_IMPORT_DESCRIPTOR   00000001800080e8     kernel32:KERNEL32.dll
 0003:000004b0       _Init_global_epoch         00000001800094b0     MSVCRT:thread_safe_statics.obj
 0003:000004c0       __security_cookie          00000001800094c0     MSVCRT:gs_cookie.obj
 0003:000004c8       __security_cookie_complement 00000001800094c8     MSVCRT:gs_cookie.obj
 0003:000004d0       __scrt_native_dllmain_reason 00000001800094d0     MSVCRT:utility.obj
 0003:000004d8       __isa_available            00000001800094d8     MSVCRT:cpu_disp.obj
 0003:000004dc       __isa_enabled              00000001800094dc     MSVCRT:cpu_disp.obj
 0003:000004e0       __memset_fast_string_threshold 00000001800094e0     MSVCRT:cpu_disp.obj
 0003:000004e8       __memset_nt_threshold      00000001800094e8     MSVCRT:cpu_disp.obj
 0003:000004f0       __scrt_ucrt_dll_is_in_use  00000001800094f0     MSVCRT:ucrt_stubs.obj
 0003:00000500       g_wrongHeapCallbacks       0000000180009500     libgetfldnm005.obj
 0003:00000580       g_szTagInfo                0000000180009580     libgetfldnm005.obj
 0003:000024c0       g_tagFlags                 000000018000b4c0     libgetfldnm005.obj
 0003:000028a8       g_refsToVerifyCnt          000000018000b8a8     libgetfldnm005.obj
 0003:000028ac       g_fakeUserData             000000018000b8ac     libgetfldnm005.obj
 0003:000028b0       g_tagVisitCount            000000018000b8b0     libgetfldnm005.obj
 0003:00003850       g_refsToVerify             000000018000c850     libgetfldnm005.obj
 0003:0001af50       g_userDataError            0000000180023f50     libgetfldnm005.obj
 0003:0001b0f0       ?_OptionsStorage@?1??__local_stdio_printf_options@@9@4_KA 00000001800240f0     libgetfldnm005.obj
 0003:0001b6b8       _tls_index                 00000001800246b8     MSVCRT:tlssup.obj
 0003:0001b6c0       __scrt_current_native_startup_state 00000001800246c0     MSVCRT:utility.obj
 0003:0001b6c8       __scrt_native_startup_lock 00000001800246c8     MSVCRT:utility.obj
 0003:0001b708       __scrt_debugger_hook_flag  0000000180024708     MSVCRT:utility_desktop.obj
 0003:0001b710       ?__type_info_root_node@@3U__type_info_node@@A 0000000180024710     MSVCRT:tncleanup.obj
 0003:0001b720       ?_OptionsStorage@?1??__local_stdio_scanf_options@@9@4_KA 0000000180024720     MSVCRT:default_local_stdio_options.obj
 0003:0001b728       __favor                    0000000180024728     MSVCRT:cpu_disp.obj
 0003:0001b730       __dyn_tls_init_callback    0000000180024730     <common>

 entry point at        0001:00002c20

 Static symbols

 0000:fffd9000       .debug$S                   0000000180000000     getfldnm005.exp
 0000:fffd9000       .debug$S                   0000000180000000     vcruntime:VCRUNTIME140.dll
 0000:fffd9000       .debug$S                   0000000180000000     vcruntime:VCRUNTIME140.dll
 0000:fffd9000       .debug$S                   0000000180000000     vcruntime:VCRUNTIME140.dll
 0000:fffd9000       .debug$S                   0000000180000000     vcruntime:VCRUNTIME140.dll
 0000:fffd9000       .debug$S                   0000000180000000     vcruntime:VCRUNTIME140.dll
 0000:fffd9000       .debug$S                   0000000180000000     vcruntime:VCRUNTIME140.dll
 0000:fffd9000       .debug$S                   0000000180000000     vcruntime:VCRUNTIME140.dll
 0000:fffd9000       .debug$S                   0000000180000000     ucrt:api-ms-win-crt-convert-l1-1-0.dll
 0000:fffd9000       .debug$S                   0000000180000000     ucrt:api-ms-win-crt-heap-l1-1-0.dll
 0000:fffd9000       .debug$S                   0000000180000000     ucrt:api-ms-win-crt-heap-l1-1-0.dll
 0000:fffd9000       .debug$S                   0000000180000000     ucrt:api-ms-win-crt-heap-l1-1-0.dll
 0000:fffd9000       .debug$S                   0000000180000000     ucrt:api-ms-win-crt-heap-l1-1-0.dll
 0000:fffd9000       .debug$S                   0000000180000000     ucrt:api-ms-win-crt-runtime-l1-1-0.dll
 0000:fffd9000       .debug$S                   0000000180000000     ucrt:api-ms-win-crt-runtime-l1-1-0.dll
 0000:fffd9000       .debug$S                   0000000180000000     ucrt:api-ms-win-crt-runtime-l1-1-0.dll
 0000:fffd9000       .debug$S                   0000000180000000     ucrt:api-ms-win-crt-runtime-l1-1-0.dll
 0000:fffd9000       .debug$S                   0000000180000000     ucrt:api-ms-win-crt-runtime-l1-1-0.dll
 0000:fffd9000       .debug$S                   0000000180000000     ucrt:api-ms-win-crt-runtime-l1-1-0.dll
 0000:fffd9000       .debug$S                   0000000180000000     ucrt:api-ms-win-crt-runtime-l1-1-0.dll
 0000:fffd9000       .debug$S                   0000000180000000     ucrt:api-ms-win-crt-runtime-l1-1-0.dll
 0000:fffd9000       .debug$S                   0000000180000000     ucrt:api-ms-win-crt-runtime-l1-1-0.dll
 0000:fffd9000       .debug$S                   0000000180000000     ucrt:api-ms-win-crt-runtime-l1-1-0.dll
 0000:fffd9000       .debug$S                   0000000180000000     ucrt:api-ms-win-crt-runtime-l1-1-0.dll
 0000:fffd9000       .debug$S                   0000000180000000     ucrt:api-ms-win-crt-runtime-l1-1-0.dll
 0000:fffd9000       .debug$S                   0000000180000000     ucrt:api-ms-win-crt-runtime-l1-1-0.dll
 0000:fffd9000       .debug$S                   0000000180000000     ucrt:api-ms-win-crt-runtime-l1-1-0.dll
 0000:fffd9000       .debug$S                   0000000180000000     ucrt:api-ms-win-crt-runtime-l1-1-0.dll
 0000:fffd9000       .debug$S                   0000000180000000     ucrt:api-ms-win-crt-runtime-l1-1-0.dll
 0000:fffd9000       .debug$S                   0000000180000000     ucrt:api-ms-win-crt-stdio-l1-1-0.dll
 0000:fffd9000       .debug$S                   0000000180000000     ucrt:api-ms-win-crt-stdio-l1-1-0.dll
 0000:fffd9000       .debug$S                   0000000180000000     ucrt:api-ms-win-crt-stdio-l1-1-0.dll
 0000:fffd9000       .debug$S                   0000000180000000     ucrt:api-ms-win-crt-stdio-l1-1-0.dll
 0000:fffd9000       .debug$S                   0000000180000000     ucrt:api-ms-win-crt-stdio-l1-1-0.dll
 0000:fffd9000       .debug$S                   0000000180000000     ucrt:api-ms-win-crt-stdio-l1-1-0.dll
 0000:fffd9000       .debug$S                   0000000180000000     ucrt:api-ms-win-crt-stdio-l1-1-0.dll
 0000:fffd9000       .debug$S                   0000000180000000     ucrt:api-ms-win-crt-stdio-l1-1-0.dll
 0000:fffd9000       .debug$S                   0000000180000000     ucrt:api-ms-win-crt-stdio-l1-1-0.dll
 0000:fffd9000       .debug$S                   0000000180000000     ucrt:api-ms-win-crt-stdio-l1-1-0.dll
 0000:fffd9000       .debug$S                   0000000180000000     ucrt:api-ms-win-crt-string-l1-1-0.dll
 0000:fffd9000       .debug$S                   0000000180000000     ucrt:api-ms-win-crt-string-l1-1-0.dll
 0000:fffd9000       .debug$S                   0000000180000000     ucrt:api-ms-win-crt-string-l1-1-0.dll
 0000:fffd9000       .debug$S                   0000000180000000     ucrt:api-ms-win-crt-string-l1-1-0.dll
 0000:fffd9000       .debug$S                   0000000180000000     ucrt:api-ms-win-crt-string-l1-1-0.dll
 0000:fffd9000       .debug$S                   0000000180000000     ucrt:api-ms-win-crt-string-l1-1-0.dll
 0000:fffd9000       .debug$S                   0000000180000000     ucrt:api-ms-win-crt-string-l1-1-0.dll
 0000:fffd9000       .debug$S                   0000000180000000     ucrt:api-ms-win-crt-string-l1-1-0.dll
 0000:fffd9000       .debug$S                   0000000180000000     kernel32:KERNEL32.dll
 0000:fffd9000       .debug$S                   0000000180000000     kernel32:KERNEL32.dll
 0000:fffd9000       .debug$S                   0000000180000000     kernel32:KERNEL32.dll
 0000:fffd9000       .debug$S                   0000000180000000     kernel32:KERNEL32.dll
 0000:fffd9000       .debug$S                   0000000180000000     kernel32:KERNEL32.dll
 0000:fffd9000       .debug$S                   0000000180000000     kernel32:KERNEL32.dll
 0000:fffd9000       .debug$S                   0000000180000000     kernel32:KERNEL32.dll
 0000:fffd9000       .debug$S                   0000000180000000     kernel32:KERNEL32.dll
 0000:fffd9000       .debug$S                   0000000180000000     kernel32:KERNEL32.dll
 0000:fffd9000       .debug$S                   0000000180000000     kernel32:KERNEL32.dll
 0000:fffd9000       .debug$S                   0000000180000000     kernel32:KERNEL32.dll
 0000:fffd9000       .debug$S                   0000000180000000     kernel32:KERNEL32.dll
 0000:fffd9000       .debug$S                   0000000180000000     kernel32:KERNEL32.dll
 0000:fffd9000       .debug$S                   0000000180000000     kernel32:KERNEL32.dll
 0000:fffd9000       .debug$S                   0000000180000000     kernel32:KERNEL32.dll
 0000:fffd9000       .debug$S                   0000000180000000     kernel32:KERNEL32.dll
 0000:fffd9000       .debug$S                   0000000180000000     kernel32:KERNEL32.dll
 0000:fffd9000       .debug$S                   0000000180000000     kernel32:KERNEL32.dll
 0000:fffd9000       .debug$S                   0000000180000000     kernel32:KERNEL32.dll
 0000:fffd9000       .debug$S                   0000000180000000     kernel32:KERNEL32.dll
 0000:fffd9000       .debug$S                   0000000180000000     kernel32:KERNEL32.dll
 0000:fffd9000       .debug$S                   0000000180000000     kernel32:KERNEL32.dll
 0000:fffd9000       .debug$S                   0000000180000000     kernel32:KERNEL32.dll
 0000:fffd9000       .debug$S                   0000000180000000     kernel32:KERNEL32.dll
 0000:fffd9000       .debug$S                   0000000180000000     kernel32:KERNEL32.dll
 0000:fffd9000       .debug$S                   0000000180000000     kernel32:KERNEL32.dll
 0000:fffd9000       .debug$S                   0000000180000000     kernel32:KERNEL32.dll
 0000:fffd9000       .debug$S                   0000000180000000     kernel32:KERNEL32.dll
 0001:00000f9c       addRefToVerify             0000000180001f9c f   libgetfldnm005.obj
 0001:00001008       agentThreadWrapper         0000000180002008 f   libgetfldnm005.obj
 0001:00001174       checkSig                   0000000180002174 f   libgetfldnm005.obj
 0001:000014a4       check_option               00000001800024a4 f   libgetfldnm005.obj
 0001:000016ec       file_basename              00000001800026ec f   libgetfldnm005.obj
 0001:00002104       startAgentThreadWrapper    0000000180003104 f   libgetfldnm005.obj
 0001:00002444       syncDebuggeeStatus         0000000180003444 f   libgetfldnm005.obj
 0001:000026e4       capture_previous_context   00000001800036e4 f   MSVCRT:gs_report.obj
 0001:00002758       ?__scrt_initialize_thread_safe_statics@@YAHXZ 0000000180003758 f   MSVCRT:thread_safe_statics.obj
 0001:00002828       ?__scrt_uninitialize_thread_safe_statics@@YAXXZ 0000000180003828 f   MSVCRT:thread_safe_statics.obj
 0001:000028d0       $$000000                   00000001800038d0     MSVCRT:amdsecgs.obj
 0001:00002900       ?dllmain_crt_dispatch@@YAHQEAUHINSTANCE__@@KQEAX@Z 0000000180003900 f   MSVCRT:dll_dllmain.obj
 0001:00002950       ?dllmain_crt_process_attach@@YAHQEAUHINSTANCE__@@QEAX@Z 0000000180003950 f   MSVCRT:dll_dllmain.obj
 0001:00002a68       ?dllmain_crt_process_detach@@YAH_N@Z 0000000180003a68 f   MSVCRT:dll_dllmain.obj
 0001:00002aec       ?dllmain_dispatch@@YAHQEAUHINSTANCE__@@KQEAX@Z 0000000180003aec f   MSVCRT:dll_dllmain.obj
 0001:00003500       $$000000                   0000000180004500     MSVCRT:guard_dispatch.obj
 0001:00003520       $$000000                   0000000180004520     MSVCRT:guard_xfg_dispatch.obj
 0001:00003536       ?fin$0@?0??dllmain_crt_process_attach@@YAHQEAUHINSTANCE__@@QEAX@Z@4HA 0000000180004536 f   MSVCRT:dll_dllmain.obj
 0001:0000354d       ?fin$0@?0??dllmain_crt_process_detach@@YAH_N@Z@4HA 000000018000454d f   MSVCRT:dll_dllmain.obj
 0001:00003566       ?fin$1@?0??dllmain_crt_process_detach@@YAH_N@Z@4HA 0000000180004566 f   MSVCRT:dll_dllmain.obj
 0001:0000357a       ?filt$0@?0??dllmain_dispatch@@YAHQEAUHINSTANCE__@@KQEAX@Z@4HA 000000018000457a f   MSVCRT:dll_dllmain.obj
 0001:000035b0       __scrt_is_nonwritable_in_current_image$filt$0 00000001800045b0 f   MSVCRT:utility.obj
 0002:00000218       ?__scrt_initialize_tss_var@@3P6AHXZEA 0000000180005218     MSVCRT:thread_safe_statics.obj
 0002:00000340       ?opcLengths@@3QBEB         0000000180005340     libgetfldnm005.obj
 0002:000022f8       GS_ExceptionPointers       00000001800072f8     MSVCRT:gs_report.obj
 0002:00002998       $unwind$fprintf            0000000180007998     libgetfldnm005.obj
 0002:000029a4       $unwind$printf             00000001800079a4     libgetfldnm005.obj
 0002:000029b0       $unwind$?NewObject@JNIEnv_@@QEAAPEAV_jobject@@PEAV_jclass@@PEAU_jmethodID@@ZZ 00000001800079b0     libgetfldnm005.obj
 0002:000029b0       $unwind$nsk_lcomplain      00000001800079b0     libgetfldnm005.obj
 0002:000029b0       $unwind$nsk_ldisplay       00000001800079b0     libgetfldnm005.obj
 0002:000029b8       $unwind$nsk_lvdisplay      00000001800079b8     libgetfldnm005.obj
 0002:000029b8       $unwind$_RTC_Initialize    00000001800079b8     MSVCRT:initsect.obj
 0002:000029b8       $unwind$_RTC_Terminate     00000001800079b8     MSVCRT:initsect.obj
 0002:000029b8       $unwind$?__scrt_initialize_thread_safe_statics@@YAHXZ 00000001800079b8     MSVCRT:thread_safe_statics.obj
 0002:000029c4       $unwind$nsk_complain       00000001800079c4     libgetfldnm005.obj
 0002:000029c4       $unwind$nsk_printf         00000001800079c4     libgetfldnm005.obj
 0002:000029cc       $unwind$nsk_lvcomplain     00000001800079cc     libgetfldnm005.obj
 0002:000029e4       $unwind$nsk_ltrace         00000001800079e4     libgetfldnm005.obj
 0002:000029e4       $unwind$__report_gsfailure 00000001800079e4     MSVCRT:gs_report.obj
 0002:000029ec       $unwind$nsk_lvtrace        00000001800079ec     libgetfldnm005.obj
 0002:000029ec       $unwind$__raise_securityfailure 00000001800079ec     MSVCRT:gs_report.obj
 0002:000029ec       $unwind$__scrt_initialize_crt 00000001800079ec     MSVCRT:utility.obj
 0002:000029ec       $unwind$__scrt_initialize_onexit_tables 00000001800079ec     MSVCRT:utility.obj
 0002:000029ec       $unwind$__scrt_release_startup_lock 00000001800079ec     MSVCRT:utility.obj
 0002:000029ec       $unwind$__scrt_uninitialize_crt 00000001800079ec     MSVCRT:utility.obj
 0002:000029ec       $unwind$_onexit            00000001800079ec     MSVCRT:utility.obj
 0002:000029f4       $unwind$nsk_lverify        00000001800079f4     libgetfldnm005.obj
 0002:00002a04       $unwind$nsk_vprintf        0000000180007a04     libgetfldnm005.obj
 0002:00002a14       $unwind$?nsk_jni_lverify@@YAHHPEAUJNIEnv_@@HQEBDH1ZZ 0000000180007a14     libgetfldnm005.obj
 0002:00002a28       $unwind$?nsk_jni_check_exception@@YAHPEAUJNIEnv_@@QEBDH@Z 0000000180007a28     libgetfldnm005.obj
 0002:00002a44       $unwind$nsk_jvmti_parseOptions 0000000180007a44     libgetfldnm005.obj
 0002:00002a60       $unwind$nsk_jvmti_createJVMTIEnv 0000000180007a60     libgetfldnm005.obj
 0002:00002a74       $unwind$Java_nsk_jvmti_unit_FollowReferences_FollowRefObjects_resetTags 0000000180007a74     libgetfldnm005.obj
 0002:00002a74       $unwind$addRefToVerify     0000000180007a74     libgetfldnm005.obj
 0002:00002a74       $unwind$nsk_jvmti_resetAgentData 0000000180007a74     libgetfldnm005.obj
 0002:00002a74       $unwind$nsk_jvmti_setFailStatus 0000000180007a74     libgetfldnm005.obj
 0002:00002a74       $unwind$__scrt_initialize_default_local_stdio_options 0000000180007a74     MSVCRT:default_local_stdio_options.obj
 0002:00002a74       $unwind$?dllmain_crt_dispatch@@YAHQEAUHINSTANCE__@@KQEAX@Z 0000000180007a74     MSVCRT:dll_dllmain.obj
 0002:00002a74       $unwind$DllMain            0000000180007a74     MSVCRT:dll_dllmain_stub.obj
 0002:00002a74       $unwind$__GSHandlerCheck   0000000180007a74     MSVCRT:gshandler.obj
 0002:00002a74       $unwind$?__scrt_uninitialize_thread_safe_statics@@YAXXZ 0000000180007a74     MSVCRT:thread_safe_statics.obj
 0002:00002a74       $unwind$__scrt_acquire_startup_lock 0000000180007a74     MSVCRT:utility.obj
 0002:00002a74       $unwind$__scrt_dllmain_after_initialize_c 0000000180007a74     MSVCRT:utility.obj
 0002:00002a74       $unwind$__scrt_dllmain_before_initialize_c 0000000180007a74     MSVCRT:utility.obj
 0002:00002a74       $unwind$__scrt_dllmain_crt_thread_attach 0000000180007a74     MSVCRT:utility.obj
 0002:00002a74       $unwind$__scrt_dllmain_crt_thread_detach 0000000180007a74     MSVCRT:utility.obj
 0002:00002a74       $unwind$__scrt_dllmain_uninitialize_c 0000000180007a74     MSVCRT:utility.obj
 0002:00002a74       $unwind$__scrt_dllmain_uninitialize_critical 0000000180007a74     MSVCRT:utility.obj
 0002:00002a74       $unwind$atexit             0000000180007a74     MSVCRT:utility.obj
 0002:00002a7c       $unwind$nsk_jvmti_lverify  0000000180007a7c     libgetfldnm005.obj
 0002:00002a90       $unwind$exitOnError        0000000180007a90     libgetfldnm005.obj
 0002:00002aa0       $unwind$check_option       0000000180007aa0     libgetfldnm005.obj
 0002:00002aa0       $unwind$_DllMainCRTStartup 0000000180007aa0     MSVCRT:dll_dllmain.obj
 0002:00002ab0       $unwind$Java_nsk_share_jvmti_ArgumentHandler_getAgentOptionsString 0000000180007ab0     libgetfldnm005.obj
 0002:00002ac4       $unwind$Java_nsk_jvmti_unit_FollowReferences_FollowRefObjects_getTag 0000000180007ac4     libgetfldnm005.obj
 0002:00002ac4       $unwind$Java_nsk_share_jvmti_DebugeeClass_checkStatus 0000000180007ac4     libgetfldnm005.obj
 0002:00002ac4       $unwind$agentThreadWrapper 0000000180007ac4     libgetfldnm005.obj
 0002:00002ad4       $unwind$Java_nsk_jvmti_GetFieldName_getfldnm005_check 0000000180007ad4     libgetfldnm005.obj
 0002:00002ad4       $unwind$startAgentThreadWrapper 0000000180007ad4     libgetfldnm005.obj
 0002:00002af0       $unwind$syncDebuggeeStatus 0000000180007af0     libgetfldnm005.obj
 0002:00002af0       $unwind$__scrt_dllmain_exception_filter 0000000180007af0     MSVCRT:utility.obj
 0002:00002b04       $unwind$Java_nsk_share_jvmti_DebugeeClass_resetAgentData 0000000180007b04     libgetfldnm005.obj
 0002:00002b0c       $unwind$Agent_Initialize   0000000180007b0c     libgetfldnm005.obj
 0002:00002b0c       $unwind$MA_checkStatus     0000000180007b0c     libgetfldnm005.obj
 0002:00002b20       $unwind$Java_nsk_jvmti_unit_FollowReferences_FollowRefObjects_setTag 0000000180007b20     libgetfldnm005.obj
 0002:00002b38       $unwind$Java_nsk_jvmti_unit_FollowReferences_FollowRefObjects_addRefToVerify 0000000180007b38     libgetfldnm005.obj
 0002:00002b54       $unwind$checkSig           0000000180007b54     libgetfldnm005.obj
 0002:00002b70       $unwind$capture_previous_context 0000000180007b70     MSVCRT:gs_report.obj
 0002:00002b7c       $unwind$__GSHandlerCheckCommon 0000000180007b7c     MSVCRT:gshandler.obj
 0002:00002b88       $xdatasym                  0000000180007b88     MSVCRT:amdsecgs.obj
 0002:00002b8c       $unwind$?dllmain_crt_process_attach@@YAHQEAUHINSTANCE__@@QEAX@Z 0000000180007b8c     MSVCRT:dll_dllmain.obj
 0002:00002bc8       $unwind$?fin$0@?0??dllmain_crt_process_attach@@YAHQEAUHINSTANCE__@@QEAX@Z@4HA 0000000180007bc8     MSVCRT:dll_dllmain.obj
 0002:00002bc8       $unwind$?fin$0@?0??dllmain_crt_process_detach@@YAH_N@Z@4HA 0000000180007bc8     MSVCRT:dll_dllmain.obj
 0002:00002bc8       $unwind$?fin$1@?0??dllmain_crt_process_detach@@YAH_N@Z@4HA 0000000180007bc8     MSVCRT:dll_dllmain.obj
 0002:00002bd0       $unwind$?dllmain_crt_process_detach@@YAH_N@Z 0000000180007bd0     MSVCRT:dll_dllmain.obj
 0002:00002c24       $unwind$?dllmain_dispatch@@YAHQEAUHINSTANCE__@@KQEAX@Z 0000000180007c24     MSVCRT:dll_dllmain.obj
 0002:00002c4c       $unwind$?filt$0@?0??dllmain_dispatch@@YAHQEAUHINSTANCE__@@KQEAX@Z@4HA 0000000180007c4c     MSVCRT:dll_dllmain.obj
 0002:00002c54       $unwind$__scrt_is_nonwritable_in_current_image 0000000180007c54     MSVCRT:utility.obj
 0002:00002c74       $unwind$__scrt_is_nonwritable_in_current_image$filt$0 0000000180007c74     MSVCRT:utility.obj
 0002:00002c7c       $unwind$__scrt_fastfail    0000000180007c7c     MSVCRT:utility_desktop.obj
 0002:00002c8c       $unwind$__security_init_cookie 0000000180007c8c     MSVCRT:gs_support.obj
 0002:00002c98       $unwind$__isa_available_init 0000000180007c98     MSVCRT:cpu_disp.obj
 0002:00002ca8       $xdatasym                  0000000180007ca8     MSVCRT:guard_dispatch.obj
 0002:00002cb0       $xdatasym                  0000000180007cb0     MSVCRT:guard_xfg_dispatch.obj
 0002:00002cc0       .edata                     0000000180007cc0     getfldnm005.exp
 0002:00002ce8       rgpv                       0000000180007ce8     getfldnm005.exp
 0002:00002d24       rgszName                   0000000180007d24     getfldnm005.exp
 0002:00002d60       rgwOrd                     0000000180007d60     getfldnm005.exp
 0002:00002d7e       szName                     0000000180007d7e     getfldnm005.exp
 0002:00002d8e       $N00001                    0000000180007d8e     getfldnm005.exp
 0002:00002d9d       $N00002                    0000000180007d9d     getfldnm005.exp
 0002:00002daa       $N00003                    0000000180007daa     getfldnm005.exp
 0002:00002dd8       $N00004                    0000000180007dd8     getfldnm005.exp
 0002:00002e1d       $N00005                    0000000180007e1d     getfldnm005.exp
 0002:00002e5a       $N00006                    0000000180007e5a     getfldnm005.exp
 0002:00002ea2       $N00007                    0000000180007ea2     getfldnm005.exp
 0002:00002ee2       $N00008                    0000000180007ee2     getfldnm005.exp
 0002:00002f1f       $N00009                    0000000180007f1f     getfldnm005.exp
 0002:00002f5a       $N00010                    0000000180007f5a     getfldnm005.exp
 0002:00002f88       $N00011                    0000000180007f88     getfldnm005.exp
 0002:00002fb9       $N00012                    0000000180007fb9     getfldnm005.exp
 0002:00002fe8       $N00013                    0000000180007fe8     getfldnm005.exp
 0002:00003017       $N00014                    0000000180008017     getfldnm005.exp
 0002:0000304c       $N00015                    000000018000804c     getfldnm005.exp
 0002:000034b2       .idata$6                   00000001800084b2     kernel32:KERNEL32.dll
 0002:00003516       .idata$6                   0000000180008516     vcruntime:VCRUNTIME140.dll
 0002:000036a8       .idata$6                   00000001800086a8     ucrt:api-ms-win-crt-heap-l1-1-0.dll
 0002:000036c8       .idata$6                   00000001800086c8     ucrt:api-ms-win-crt-runtime-l1-1-0.dll
 0002:000036ea       .idata$6                   00000001800086ea     ucrt:api-ms-win-crt-convert-l1-1-0.dll
 0002:0000370c       .idata$6                   000000018000870c     ucrt:api-ms-win-crt-stdio-l1-1-0.dll
 0002:0000372c       .idata$6                   000000018000872c     ucrt:api-ms-win-crt-string-l1-1-0.dll
 0003:00000000       ?codeAttributeName@@3PEBDEB 0000000180009000     libgetfldnm005.obj
 0003:00000008       ?lineNumberAttributeName@@3PEBDEB 0000000180009008     libgetfldnm005.obj
 0003:00000010       ?localVarAttributeName@@3PEBDEB 0000000180009010     libgetfldnm005.obj
 0003:00000018       ?localVarTypeAttributeName@@3PEBDEB 0000000180009018     libgetfldnm005.obj
 0003:00000020       ?stackMapAttributeName@@3PEBDEB 0000000180009020     libgetfldnm005.obj
 0003:00000028       ?callBytes@@3PAEA          0000000180009028     libgetfldnm005.obj
 0003:0000002c       ?allocBytes@@3PAEA         000000018000902c     libgetfldnm005.obj
 0003:00000030       fld_sig                    0000000180009030     libgetfldnm005.obj
 0003:0001af54       redefineAttempted          0000000180023f54     libgetfldnm005.obj
 0003:0001af58       nsk_context                0000000180023f58     libgetfldnm005.obj
 0003:0001af64       redefineSucceed            0000000180023f64     libgetfldnm005.obj
 0003:0001af68       agentFailed                0000000180023f68     libgetfldnm005.obj
 0003:0001af6c       currentAgentStatus         0000000180023f6c     libgetfldnm005.obj
 0003:0001af70       context                    0000000180023f70     libgetfldnm005.obj
 0003:0001b028       agentThread                0000000180024028     libgetfldnm005.obj
 0003:0001b030       agentThreadProc            0000000180024030     libgetfldnm005.obj
 0003:0001b038       agentThreadArg             0000000180024038     libgetfldnm005.obj
 0003:0001b040       agent_data                 0000000180024040     libgetfldnm005.obj
 0003:0001b050       jvmti_env                  0000000180024050     libgetfldnm005.obj
 0003:0001b058       jvm                        0000000180024058     libgetfldnm005.obj
 0003:0001b060       jni_env                    0000000180024060     libgetfldnm005.obj
 0003:0001b068       checkStatus_func           0000000180024068     libgetfldnm005.obj
 0003:0001b070       ?codeAttributeIndex@@3GA   0000000180024070     libgetfldnm005.obj
 0003:0001b074       ?lineNumberAttributeIndex@@3GA 0000000180024074     libgetfldnm005.obj
 0003:0001b078       ?localVarAttributeIndex@@3GA 0000000180024078     libgetfldnm005.obj
 0003:0001b07c       ?localVarTypeAttributeIndex@@3GA 000000018002407c     libgetfldnm005.obj
 0003:0001b080       ?stackMapAttributeIndex@@3GA 0000000180024080     libgetfldnm005.obj
 0003:0001b084       ?stackFrameOffset@@3GA     0000000180024084     libgetfldnm005.obj
 0003:0001b088       ?mode@@3HA                 0000000180024088     libgetfldnm005.obj
 0003:0001b08c       ?constantPoolSize@@3GA     000000018002408c     libgetfldnm005.obj
 0003:0001b090       ?orig@@3PEBEEB             0000000180024090     libgetfldnm005.obj
 0003:0001b098       ?gen@@3PEAEEA              0000000180024098     libgetfldnm005.obj
 0003:0001b0a0       ?inputPos@@3PEAEEA         00000001800240a0     libgetfldnm005.obj
 0003:0001b0a8       ?endPos@@3PEBEEB           00000001800240a8     libgetfldnm005.obj
 0003:0001b0b0       ?genPos@@3PEAEEA           00000001800240b0     libgetfldnm005.obj
 0003:0001b0b8       ?markPos@@3PEAEEA          00000001800240b8     libgetfldnm005.obj
 0003:0001b0c0       ?constantPool@@3PEAPEADEA  00000001800240c0     libgetfldnm005.obj
 0003:0001b0c8       ?constantPoolCount@@3GA    00000001800240c8     libgetfldnm005.obj
 0003:0001b0cc       ?zeroBytes@@3PAEA          00000001800240cc     libgetfldnm005.obj
 0003:0001b0d0       ?codeLength@@3IA           00000001800240d0     libgetfldnm005.obj
 0003:0001b0d8       ?map@@3PEAIEA              00000001800240d8     libgetfldnm005.obj
 0003:0001b0e0       ?widening@@3PEACEA         00000001800240e0     libgetfldnm005.obj
 0003:0001b0e8       jvmti                      00000001800240e8     libgetfldnm005.obj
 0003:0001b100       GS_ExceptionRecord         0000000180024100     MSVCRT:gs_report.obj
 0003:0001b1a0       GS_ContextRecord           00000001800241a0     MSVCRT:gs_report.obj
 0003:0001b670       ?g_tss_cv@@3U_RTL_CONDITION_VARIABLE@@A 0000000180024670     MSVCRT:thread_safe_statics.obj
 0003:0001b678       ?g_tss_event@@3PEAXEA      0000000180024678     MSVCRT:thread_safe_statics.obj
 0003:0001b680       ?g_tss_mutex@@3U_RTL_CRITICAL_SECTION@@A 0000000180024680     MSVCRT:thread_safe_statics.obj
 0003:0001b6a8       ?g_sleep_condition_variable_cs@@3P6AHPEAU_RTL_CONDITION_VARIABLE@@PEAU_RTL_CRITICAL_SECTION@@K@ZEA 00000001800246a8     MSVCRT:thread_safe_statics.obj
 0003:0001b6b0       ?g_wake_all_condition_variable@@3P6AXPEAU_RTL_CONDITION_VARIABLE@@@ZEA 00000001800246b0     MSVCRT:thread_safe_statics.obj
 0003:0001b6bc       ?__proc_attached@@3HA      00000001800246bc     MSVCRT:dll_dllmain.obj
 0003:0001b6d0       ?is_initialized_as_dll@@3_NA 00000001800246d0     MSVCRT:utility.obj
 0003:0001b6d1       ?module_local_atexit_table_initialized@@3_NA 00000001800246d1     MSVCRT:utility.obj
 0003:0001b6d8       ?module_local_atexit_table@@3U_onexit_table_t@@A 00000001800246d8     MSVCRT:utility.obj
 0003:0001b6f0       ?module_local_at_quick_exit_table@@3U_onexit_table_t@@A 00000001800246f0     MSVCRT:utility.obj
